:020000020000FC
:0200000009C035
:10000C007FB76A957FBF1895EFEDEDBFE8E0E7BBD2
:10001C00E5E0E3BFE2E0E9BF7894E0E4EFBDE9E0BE
:10002C00EEBD4427F2E0EAE2042E000CE00D43950D
:10003C00C895502DE395C89507FC0DC0602DF2E0D6
:10004C00E0E0550FE50FC8950ABCE395C8950BBCCD
:0E005C006623F1F7E7CFEFE3E5BF8895D5CF38
:10020000642C34286A24FB20DF1D0E1B8118321653
:100210001A1435127E10F00E870D410C190B0D0AC1
:100220001A093F087807C4062006011002100310BF
:100230000410051006100710081009100A100B1002
:100240000C100D100E100D200B200920072005208A
:06025000032001200080E4
:00000001FF
